:20FFD600E000E000E000E000E000E000E000E000E000E000E000E000E000FD00E000E000EE
:0AFFF600E000E000E000E000E000A1
:20C00000464C094B5420202020005350454349414C50524F472E3F20202000535045432E07
:20C0200050524F47204B4C41523F200050524F4752414D46454C00000000000000414E475A
:20C0400045204B4F443A00000000000000007300204E31202020204E32202020204E332030
:20C0600000492F4F20544553543F00494E47084E4720414B542E3A00555447084E47204189
:20C080004B542E3A0046454C484953544F52494B3F2020202000414E542E50524F472E3AE5
:20C0A000000050554D505449443A0000000044524946545241444552494E472021212000DC
:20C0C00054454D502031204F46465345543A0054454D502032204F46465345543A00736537
:20C0E0006B006D003F002E0050524F4752414D4D4552494E4720202000202000DF43006DF2
:20C10000696E00204D4544202000205554414E200050002000300025006800094E4452413F
:20C12000204B4F443A0000000000000042525954205354520A4D4D454E000000004D415256
:20C140004B45524120494E53502E3F2020005609524D455220534B0A4C4A54414E4B00474D
:20C1600052414E554C4154004449534B415220202000534B0A4C4A45522020005649444151
:20C180005245203D2053544152542020005354094E4720440A5252415220460A520056417A
:20C1A0005454454E46594C4C4E494E4720200046594C4C45522056415454454E2020200081
:20C1C00044524946544B4C4152202020202020200046454C2046594C4C4E494E4720202022
:20C1E000200050524F562050524F4752414D20202020005354094E4720440A525241524EE8
:20C20000412020002020202053544F50504144202020202000202020202020202020202002
:20C2200020202020200046454C2053094B4552482E4E495608200046454C2053094B42526C
:20C24000595441524520200046454C204D4F544F52534B59444420200046454C200A482D5C
:20C26000534B594444202020200046454C2056415454454E545259434B20005354415254BB
:20C280003D4A412020203F3D4E454A004C41444441205354414E444152443F20004C414426
:20C2A0004441205354414E444152443F3F00414E54414C2050524F4752414D3A0000002008
:20C2C0004449534B544944202000000000000000094E445241200A56524947413F202020A2
:20C2E00000534B0A4C4A54454D503A000000000000004449534B54454D503A0000000000F5
:20C3000000000053455041524154494F4E3A000000000000534B0A4C4A5449443A00000094
:20C3200000000000004E495608204449534B3A000000000000004E49560820534B0A4C4A30
:20C340003A000000000000464C094B54205449443A00000000000000534B0A4C4A4D45441A
:20C36000454C000000000000004B4C4152200A565249474120202020200050524F475241F4
:20C380004D4D2E204B4C4152202000454E474C4953483F20202020202020200044455554D0
:20C3A0005343483F2020202020202020004652414E434149533F2020202020202000535651
:20C3C000454E534B413F20202020202020200053554F4D493F2020202020202020202000A0
:20C3E0004E454445524C414E44533F2020202020004954414C49414E4F3F2020202020202E
:20C4000020004E4F52534B3F2020202020202020202000455350414E4F4C3F2020202020FF
:15C420002020200044414E534B3F2020202020202020202000B7
:20C4600046414E202020202020005350454349414C2050524F472E3F202000535045432EC8
:20C4800050524F472E204F4B3F20200050524F4752414D204552524F5200000000494E5054
:20C4A000555420434F44453A0000000000007300204E31202020204E32202020204E33202B
:20C4C00000492F4F20544553543F00494E47084E4720414B542E3A00555447084E47204125
:20C4E0004B542E3A004552524F52204D455353414745532020004E4F2E50524F473A0000B6
:20C50000000050554D5054494D453A00000044524946545241444552494E47202121200029
:20C5200054454D502031204F46465345543A0054454D502032204F46465345543A007365D2
:20C5400063006D003F002E0050524F4752414D4D494E47202020202000202000DF43006DEC
:20C56000696E002057495448200020572F4F202000500020003000250068004348414E47A5
:20C580004520434F44453A00000000005455524E204D414348494E45204F4646004D4152A8
:20C5A0004B20494E5350454354494F4E3F0048454154494E4720424F494C45522020004771
:20C5C00052414E554C4553005741534845532020200052494E53455320202000434F4E54AE
:20C5E000494E5545203D20535441525400434C4F534520444F4F5220464F52202000574156
:20C600005445522D46494C4C494E472020200046494C4C53205741544552202020202000E0
:20C62000524541445920544F2057415348202020004552524F522046494C4C494E47202020
:20C640002000545249414C2050524F4752414D4D452000434C4F534520444F4F52532020F7
:20C6600020202000202020494E544552555054454420202000202020202020202020202036
:20C680002020202020004552524F522053414645204C4556454C004552524F522053414615
:20C6A00045545953572E20004552524F52204D4F544F5250524F5420004552524F522053F3
:20C6C000555045524850524F54004552524F52205741544552505245535300535441525449
:20C6E0003D5945532020203F3D4E4F004C4F4144204445462E56414C5545533F004C4F416B
:20C7000044204445462E56414C5545533F004E4F2E4F462050524F47522E3A000000002017
:20C720005741534854494D4520000000000000004348414E4745204F54482E56414C3F2056
:20C740000052494E53452D54454D503A000000000000574153482D54454D503A00000000EB
:20C7600000000053455041524154494F4E3A00000000000052494E53452D54494D453A0072
:20C7800000000000004C4556454C20574153483A0000000000004C4556454C20424F494CD6
:20C7A00045523A0000000046414E2054494D453A000000000000000052494E534520414721
:20C7C000454E5400000000000046494E4953484544204F54482E56414C0050524F47522E54
:20C7E0002046494E49534845442000454E474C4953483F2020202020202020004445555434
:20C800005343483F2020202020202020004652414E434149533F20202020202020005356EC
:20C82000454E534B413F20202020202020200053554F4D493F20202020202020202020003B
:20C840004E454445524C414E44533F2020202020004954414C49414E4F3F202020202020C9
:20C8600020004E4F52534B3F2020202020202020202000455350414E4F4C3F20202020209B
:15C880002020200044414E534B3F202020202020202020200053
:20C8C0004C0E46544552202020005350455A49414C2050524F472E3F2020005350455A2EE0
:20C8E00050524F472E204F4B3F20200050524F4752414D4D204645484C45520000434F4488
:20C90000452045494E474542454E3A0000007300204E31202020204E32202020204E332008
:20C9200000492F4F20544553543F00494E47084E4720414B542E3A00555447084E472041C0
:20C940004B542E3A004645484C45524D454C44554E47454E2000414E5A2E50524F472E3AA4
:20C96000000050554D504544415545523A0044524946545241444552494E4720212120003E
:20C9800054454D502031204F46465345543A0054454D502032204F46465345543A0073656E
:20C9A0006B006D003F002E0050524F4752414D4D494552554E47202000202000DF43004D14
:20C9C000696E00204D4954202000204F484E452000500020003000250068004E4555455220
:20C9E00020434F44453A0000000000005354524F4D2041425354454C4C454E0000494E5389
:20CA0000502E204D41524B4945522E3F2000484549545A5420424F494C4552202020004784
:20CA200052414E554C41540053500E4C454E202020004B4C415253500E4C2000574549546F
:20CA40004552203D205354415254202000540E5245205343484C49455353454E2000460E76
:20CA60005220574153534552460E4C4C454E00460E4C4C542057415353455220202020003B
:20CA800042455452494542534245524549542020004645484C455220460E4C4C454E2020B6
:20CAA0002000564552535543482050524F4752414D4D00540E5245205343484C494553533A
:20CAC000454E20002050524F4752414D4D53544F50502020002020202020202020202020E8
:20CAE0002020202020004645484C2E534943482E4E4956454155004645484C2E53494348B8
:20CB00002E534348414C54004645484C2E204D4F544F525343482E20004645484C200E4869
:20CB20002D53434855545A2020004645484C2E574153534552445255434B0053544152547E
:20CB40003D4A4120203F3D4E45494E005745524B5357455254204C4144454E3F00574552A8
:20CB60004B5357455254204C4144454E3F00414E5A2E2050524F4752414D4D3A000000201C
:20CB800053500E4C5A4549542000000000000000414E442E574552544520094E44524E3F1A
:20CBA000004B4C415253500E4C544D503A000000000053500E4C54454D503A0000000000B6
:20CBC00000000041425452454E4E44415545523A000000004B4C415253500E4C444155524D
:20CBE0003A000000004E49562E2053500E4C454E3A00000000004E49562E20424F494C4550
:20CC0000523A00000000004C0E4654455244415545523A00000000004B4C415253502E4D0A
:20CC200049544C000000000000414E44455245205745525445204F4B3F0050524F475241F1
:20CC40004D2E204645525449473F00454E474C4953483F20202020202020200044455554BE
:20CC60005343483F2020202020202020004652414E434149533F2020202020202000535688
:20CC8000454E534B413F20202020202020200053554F4D493F2020202020202020202000D7
:20CCA0004E454445524C414E4453202020202020004954414C49414E4F3F20202020202084
:20CCC00020004E4F52534B3F2020202020202020202000455350414E4F4C3F202020202037
:15CCE0002020200044414E534B3F2020202020202020202000EF
:20CD200056454E54494C4552200050524F472E205350454349414C453F200050524F472ED9
:20CD400020535045432E204F4B3F200050524F4752414D4D452045525245555200494E53B8
:20CD60004552455220434F44453A000000007300204E31202020204E32202020204E3320DD
:20CD800000492F4F20544553543F00494E47084E4720414B542E3A00555447084E4720415C
:20CDA0004B542E3A00414646495343482E2045525245555220004E425245205047522E3A9D
:20CDC00000004455520B4520504D503A000044524946545241444552494E4720212120008A
:20CDE00054454D502031204F46465345543A0054454D502032204F46465345543A0073650A
:20CE000063006D003F002E0050524F4752414D4D4154494F4E20202000202000DF43006DC6
:20CE2000696E00204156454320002053414E532000500020003000250068004E4F5556458D
:20CE4000415520434F44453A00000000455441494E445245204D4143482E000000504F492C
:20CE60004E54204420494E53504543542E004D495345200D2054454D5020424F552E00471C
:20CE800052414E554C4553004C41564520202020200052494E43452020202000434F4E548B
:20CEA000494E5545203D205354415254004645524D455420504F525445532050520052451D
:20CEC0004D504C49535341474520454155200052454D504C495420454155202020202000DA
:20CEE00050520C5445204155204C415641474520004552524555522052454D504C495353E1
:20CF00002E005047522E204558504552494D454E5420004645524D455420504F52544553CB
:20CF20002020200020202020204152520C542020202020200020202020202020202020208C
:20CF40002020202020004552522E4E4956454155205345435552004552522E494E54455217
:20CF600052205345435552004552522E5345435552204D4F54455552004552522E20534559
:20CF800055522053555243482E004552522E2050524553532045415520200053544152548A
:20CFA0003D4F554920203F3D4E4F4E0056414C2E4445462E205553494E453F200056414CAC
:20CFC0002E4445462E205553494E453F3F004E4252452044452050524F47522E3A00002002
:20CFE0004455522E4C41562E20000000000000004348414E474520415554522056414C3FA3
:20D0000000544D502052494E0F4147453A000000000054454D50204C41564147453A0000C0
:20D020000000004455522E20534550415241543A000000004455522E2052494E0F4147456F
:20D040003A000000004E49562E204C41564147453A00000000004E49562E20424F55494CBB
:20D060004C3A00000000004455522E56454E54494C2E3A00000000004147454E54205249AD
:20D080004E0F2E00000000000050520C54204155545245533F202020200050524F47522E98
:20D0A0005445524D494E0B453F2000454E474C4953483F2020202020202020004445555477
:20D0C0005343483F2020202020202020004652414E434149533F2020202020202000535624
:20D0E000454E534B413F20202020202020200053554F4D493F202020202020202020200073
:20D100004E454445524C414E44533F2020202020004954414C49414E4F3F20202020202000
:20D1200020004E4F52534B3F2020202020202020202000455350414E4F4C3F2020202020D2
:15D140002020200044414E534B3F20202020202020202020008A
:20D18000505548414C4C494E20004552494B4F49534F484A2E3F20202020004F484A454CBC
:20D1A0004D4F494E5449204F4B3F20004F484A454C4D4156495248452000000000414E4E0B
:20D1C00041204B4F4F44493A0000000000007300204E31202020204E32202020204E33200B
:20D1E00000492F4F20544553543F00494E47084E4720414B542E3A00555447084E472041F8
:20D200004B542E3A0056494B41484953544F52494120202020004F484A454C2E4C4B4D3A3B
:20D22000000050554D50505541494B3A000044524946545241444552494E472021212000B1
:20D2400054454D502031204F46465345543A0054454D502032204F46465345543A007365A5
:20D260006B006D003F002E004F484A454C4D4F494E5449202020202000202000DF43004DD8
:20D28000494E00202B2020202000202D2020202000500020003000250068005641494844C6
:20D2A00041204B4F4F44493A000000004B41544B414953452056495254413A00004B49524A
:20D2C0004A41205441524B49535455533F0048555548542E564544454E204C094D4D00520B
:20D2E0004145504553552000504553552020202020004855554854454C5520004A41544BB0
:20D3000041203D2053544152542020200053554C4A45204F56455420202020202000564525
:20D3200044454E54095954540A202020202000540959540909205645545409202020200006
:20D340004B095954540A56414C4D4953202020200056090952092054095954540A20202077
:20D3600020004B4F454F484A454C4D412020202020200053554C4A45204F564554202020AD
:20D38000202020005649524845205059530959544554545900202020202020202020202037
:20D3A000202020202000564952484520545552564152414A412000564952484520545552C6
:20D3C00056414B59544B2E005649524845204D4F4F54544F524920200056495248452059F3
:20D3E0004C494B55554D2E202000564952484520564553495041494E4520005354415254F8
:20D400003D202B2020203F3D202D20004C415441412056414B494F3F20202020004C41549E
:20D4200041412056414B494F3F3F202020004F484A454C4D49454E204C4B4D3A00000020F9
:20D440005045535541492E3A20000000000000004D55555441204D555554203F20202020A7
:20D460000048555548542E4C094D503A000000000000504553554C094D500A543A000000FD
:20D4800000000052454B45455420504F4C533A000000000048555548542E41494B413A0028
:20D4A0000000000000414E5455524920504553553A0000000000414E54555249204855551D
:20D4C00048543A00000000505548414C4C2E41494B413A000000000048555548542E4149EC
:20D4E0004E453A0000000000004D5555542056414C4D49533F20202020004F484A454C4DAA
:20D50000412056414C4D49533F2000454E474C4953483F2020202020202020004445555404
:20D520005343483F2020202020202020004652414E434149533F20202020202020005356BF
:20D54000454E534B413F20202020202020200053554F4D493F20202020202020202020000E
:20D560004E454445524C414E44533F2020202020004954414C49414E4F3F2020202020209C
:20D5800020004E4F52534B3F2020202020202020202000455350414E4F4C3F20202020206E
:15D5A0002020200044414E534B3F202020202020202020200026
:20D5E00056454E54494C41542000535045432E50524F472E5354414E443F00535045432ED3
:20D600002050524F472E204F4B3F200050524F4752414D4D4120464F55540000005741438C
:20D620004854574F4F52443A0000000000007300204E31202020204E32202020204E332056
:20D6400000492F4F20544553543F00494E47084E4720414B542E3A00555447084E47204193
:20D660004B542E3A00464F5554204D454C44494E47454E20200041414E542E50524F473AAE
:20D680000000504F4D5054494A443A00000044524946545241444552494E472021212000A2
:20D6A00054454D502031204F46465345543A0054454D502032204F46465345543A00736541
:20D6C00063006D003F002E0050524F4752414D4D4552454E2020202000202000DF43004D4F
:20D6E000494E00204D4554202000204745454E2000500020003000250068004E4945555739
:20D700002E5741434854573A00000000484F4F4644534348414B2E2055495400004E415AD0
:20D72000494348542050554E543F20202000564552572E20424F494C455220202020004BA1
:20D740004F5252454C53200057415353454E202020004E4153504F454C202000564552441E
:20D760004552203D20535441525420200044554552454E20534C554954454E202000564FDB
:20D780004F522056554C4C454E20202020200056554C5420574154455220202020202000A4
:20D7A0004B4C415220562E2057415353454E202000464F55542056554C2020202020202035
:20D7C0002000544553542050524F4752414D4D41202000534C5549542044455552454E204F
:20D7E0002020200050524F47522E4F4E44455242524F4B2E002020202020202020202020DD
:20D80000202020202000464F55542057415445524E495645415500464F5554204445555231
:20D82000534348414B202000504F4D50204F56455242454C415354200044524F4F474B4FB6
:20D840004F4B20424556202020004C4147452057415445524452554B202000535441525411
:20D860003D4A412020203F3D4E454500464142522E494E5354454C4C2E3F20200046414252
:20D88000522E494E5354454C4C2E3F3F200041414E542E50524F4752414D2E3A000000202F
:20D8A00057415354494A443A2000000000000000414E44455245204745472E57494A5A3FA5
:20D8C000004E4153504F4C54454D503A00000000000057415354454D503A000000000000B0
:20D8E0000000004E412057415353454E3A000000000000004E4153504F4C54494A443A003C
:20D9000000000000004E49562E2057415354414E4B3A000000004E49562E20424F494C45D3
:20D92000523A000000000056454E542E2054494A443A0000000000004E4153504F454C4D0C
:20D9400049442E000000000000414E44455245204745472E204F4B3F200050524F47524158
:20D960004D2E4B4C4141523F202000454E474C4953483F20202020202020200044455554C7
:20D980005343483F2020202020202020004652414E434149533F202020202020200053565B
:20D9A000454E534B413F20202020202020200053554F4D493F2020202020202020202000AA
:20D9C0004E454445524C414E44533F2020202020004954414C49414E4F3F20202020202038
:20D9E00020004E4F52534B3F2020202020202020202000455350414E4F4C3F20202020200A
:15DA00002020200044414E534B3F2020202020202020202000C1
:20DA800056454E544F4C4120200050524F47522E205350454349414C453F0046494E45208E
:20DAA00050524F472E535045432E3F004552524F52452050524F4752414D4D4100434F44FD
:20DAC00049434520494E5055543A000000007300204E31202020204E32202020204E332058
:20DAE00000492F4F20544553543F00494E47084E4720414B542E3A00555447084E472041EF
:20DB00004B542E3A004552524F524520202020202020202020004E522E505247523A0000AC
:20DB200000004F524520504F4D50413A000044524946545241444552494E472021212000E1
:20DB400054454D502031204F46465345543A0054454D502032204F46465345543A0073659C
:20DB600063006D003F002E0050524F4752414D4D415A494F4E45202000202000DF43004D4E
:20DB8000494E0020434F4E2020002053454E5320005000200030002500680043414D4249AC
:20DBA0004120434F442E3A0000000000535045474E49204D41434348494E410000535049C0
:20DBC0004120434F4E54524F4C4C4F3F200052495343414C444920424F494C45522000473A
:20DBE00052414E554C4920004C41564120202020200053434941435155412000434F4E54D8
:20DC0000494E554F203D2053544152540043484955444920504F52544520504552005249BC
:20DC2000454D50494D2E2041435155412020005249454D504945204143515541202020007D
:20DC40004F4B204C4156414747494F2020202020004552524F5245204C4956454C4C4F20FA
:20DC6000200050524F4752414D4D412050524F56412000434849555355524120504F52544D
:20DC800045202000202020204152524553544F20202020200020202020202020202020205F
:20DCA0002020202020004552522E204C49562E2053494355522E004552522E204D4943523E
:20DCC0004F20504F525441004552522E2050524F54455A2E4D4F542E004552522E20535509
:20DCE0005252495343414C442E004552522E2050524553532E4143515541005354415254B7
:20DD00003D5349202020203F3D4E4F0050524F4752414D4120424153453F20200050524F8D
:20DD20004752414D4120424153453F3F20004E522E2050524F4752414D4D493A00000020AC
:20DD40004455522E4C41563A20000000000000005641522E20414C5452492056414C3F2058
:20DD60000054DF20534349414351554F3A000000000054DF204C4156414747494F3A0000E7
:20DD80000000004455522E205345504152415A3A000000004455522E534349414351554F89
:20DDA0003A000000004C49562E4C4156414747494F3A000000004C49562E20424F494C45E8
:20DDC000523A00000000004455522E56454E54494C2E3A00000000004252494C4C49414E17
:20DDE000542020000000000000414C54524920564F4C4F5249204F4B3F0046494E4520508D
:20DE0000524F4752414D4D413F2000454E474C4953483F20202020202020200044455554D2
:20DE20005343483F2020202020202020004652414E434149533F20202020202020005356B6
:20DE4000454E534B413F20202020202020200053554F4D493F202020202020202020200005
:20DE60004E454445524C414E44533F2020202020004954414C49414E4F3F20202020202093
:20DE800020004E4F52534B3F2020202020202020202000455350414E4F4C3F202020202065
:15DEA0002020200044414E534B3F20202020202020202020001D
:20800000564946544520202020005350455349414C50524F472E3F20202000535045432EF3
:2080200050524F472E4B4C41523F200050524F4752414D4645494C2020202020004B4F449B
:20804000453A0000000000000000000000007300204E31202020204E32202020204E33206E
:2080600000492F4F20544553543F00494E47084E4720414B542E3A00555447084E472041C9
:208080004B542E3A004645494C484953544F52494B20202020004E522E505247523A000089
:2080A000000050554D50455449443A00000044524946545241444552494E472021212000D7
:2080C00054454D502031204F46465345543A0054454D502032204F46465345543A00736577
:2080E0006B006D003F002E0050524F4752414D4D4552494E4720202000202000DF43006D32
:20810000696E00204D4544202000205554454E200050002000300025006800454E4452453B
:20812000204B4F44453A0000000000004252595420535452304D4D454E000000004D455227
:208140004B20494E53502E3F2020202020005641524D455220534B594C4C54414E4B00477C
:2081600052414E554C4154005641534B455220202000534B594C4C4552202000564944452E
:208180005245203D2053544152542020005354454E4720444F52454E4520464F5200564101
:2081A0004E4E46594C4C4E494E47202020200046594C4C45522056414E4E2020202020007F
:2081C0004452494654534B4C4152202020202020004645494C204D45442046594C4C494EE5
:2081E00047005445535450524F4752414D2020202020005354454E4720444F52454E4520C2
:20820000202020002020202053544F5050455420202020200020202020202020202020204F
:208220002020202020004645494C2053494B4B45482E4E49562E004645494C2053494B4BE4
:208240002E425259542E20004645494C204D4F544F525645524E2020004645494C20542E53
:208260004B2E53494B522E2020004645494C2056414E4E545259434B202000535441525410
:208280003D4A412020203F3D4E4549005354442E20564552444945523F202020005354448A
:2082A0002E20564552444945523F3F202000414E54414C4C2050524F4752414D3A00002053
:2082C0005641534B5449443A2000000000000000454E44524520414E4E45543F202020206B
:2082E00000534B594C4C4554454D503A2000000000005641534B4554454D503A20200000F0
:20830000000000534550455241534A4F4E3A000000000000534B594C4C455449443A00003A
:2083200000000000004E495641205641534B3A000000000000004E49564120534B594C4CA3
:208340003A00000000000056494654455449443A0000000000000000544F5252454D4944E4
:2083600044454C0000000000004F2E4B2E20414E4E45543F20202020200050524F475241F2
:208380004D204F2E4B2E3F20202000454E474C4953483F2020202020202020004445555460
:2083A0005343483F2020202020202020004652414E434149533F2020202020202000535691
:2083C000454E534B413F20202020202020200053554F4D493F2020202020202020202000E0
:2083E0004E454445524C414E44533F2020202020004954414C49414E4F3F2020202020206E
:2084000020004E4F52534B3F2020202020202020202000455350414E4F4C3F20202020203F
:158420002020200044414E534B3F2020202020202020202000F7
:2084600056454E54494C4152200050524F472E2045535045432E3F2020200050524F472E4E
:208480002045535045432E204F4B3F004552524F522050524F4752414D41202000494E54F7
:2084A000524F20434F4449474F3A000000007300204E31202020204E32202020204E3320D9
:2084C00000492F4F20544553543F00494E47084E4720414B542E3A00555447084E47204165
:2084E0004B542E3A004D454E53414A4553204552524F522020004E522E505247523A0000F2
:2085000000004455522E424F4D42413A000044524946545241444552494E47202121200060
:2085200054454D502031204F46465345543A0054454D502032204F46465345543A00736512
:2085400063006D003F002E0050524F4752414D4D4143494F4E20202000202000DF43006DE0
:20856000696E0020434F4E2020002053494E2020005000200030002500680043414D424911
:208580004520434F442E3A0000000000415041474152204D415155494E410000004D415280
:2085A00043415220494E53504543432E3F0043414C454E54414E444F20424F494C5200479B
:2085C00052414E554C4F20004C4156414E444F20200041434C415241444F2000434F4E54DA
:2085E000494E5541523D205354415254004345525241522050554552544120202000504170
:208600005241204C4C454E4152204147554100434F4749454E444F204147554120202000C5
:208620005055454445204C415641522020202020004552524F52204C4C454E41444F2020A8
:20864000200050524F4752414D4120444520544553540043455252415220505545525441E8
:20866000202020002020494E544552555043494F4E2020200020202020202020202020204A
:208680002020202020004552522E4E4956454C2053454755522E004552522E53454E532E53
:2086A00020505545525441004552522E204D4F544F522D50524F542E004552522E50524F59
:2086C0005445432E5445524D2E004552522E50524553494F4E204147554100535441525427
:2086E0003D53492020203F3D4E4F4E00204441544F5320464142524943413F200020444133
:20870000544F5320464142524943413F3F004E522E2050524F4752414D413A00000000203C
:208720004455522E4C41563A200000000000000020434F4D422E4F54524F532056414C3F9B
:208740000054DF2041434C415241444F3A000000000054DF204C415641444F3A0000000011
:2087600000000053455041524143494F4E3A0000000000004455522E41434C415241444F8A
:208780003A000000004E49562E2054414E5155453A00000000004E49562E20424F494C45B6
:2087A000523A00000000004455522E56454E54494C2E3A000000000050524F442E204252C3
:2087C000494C4C4F0000000000204F54524F2056414C2E204F4B3F2020002046494E414C11
:2087E0002050524F4752414D413F00454E474C4953483F2020202020202020004445555446
:208800005343483F2020202020202020004652414E434149533F202020202020200053562C
:20882000454E534B413F20202020202020200053554F4D493F20202020202020202020007B
:208840004E454445524C414E44533F2020202020004954414C49414E4F3F20202020202009
:2088600020004E4F52534B3F2020202020202020202000455350414E4F4C3F2020202020DB
:158880002020200044414E534B3F202020202020202020200093
:2088C00056454E54494C415420005350454349414C50524F472E3F20202000535045432EB2
:2088E00050524F47204B4C41523F200050524F4752414D46454A4C2020202020004B4F44E0
:20890000453A0000000000000000000000007300204E31202020204E32202020204E3320A5
:2089200000492F4F20544553543F00494E47084E4720414B542E3A00555447084E47204100
:208940004B542E3A0046454A4C484953544F52494B3F20202000414E542E50524F472E3A32
:20896000000050554D50455449443A00000044524946545241444552494E4720212120000E
:2089800054454D502031204F46465345543A0054454D502032204F46465345543A007365AE
:2089A0006B006D003F002E0050524F4752414D4D4552494E4720202000202000DF43006D69
:2089C000696E00204D4544202000205544454E20005000200030002500680041454E445287
:2089E00045204B4F44453A0000000000534C554B20535452304D4D454E000000004D415220
:208A00004B455220494E53502E3F202020005641524D455220534B594C4C54414E4B00475C
:208A200052414E554C4154005641534B455220202000534B594C4C45522020005649444565
:208A40005245203D2053544152542020004C554B20443052454E4520464F522020005641AC
:208A60004E44500846594C444E494E47202000500846594C4445522056414E4E20202000A0
:208A800044524946544B4C4152202020202020200046454A4C204D2E2046594C444E494E63
:208AA00047005445535450524F4752414D2020202020004C554B20443052454E452020206D
:208AC000202020002020202053544F50504554202020202000202020202020202020202087
:208AE00020202020200046454A4C2053494B4B4552482E4E49560046454A4C20444F524BF8
:208B00004F4E54414B54200046454A4C204D4F544F52564145524E200046454A4C20542E33
:208B20004B2E53494B522E20200046454A4C2056414E445452594B20202000535441525473
:208B40003D4A412020203F3D4E454A005354442E20564552444945523F20202000535444C0
:208B60002E20564552444945523F3F202000414E54414C2050524F4752414D3A00000020D6
:208B80005641534B4554443A200000000000000041454E445245204F56524947413F202053
:208BA00000534B594C4C4554454D503A0000000000005641534B4554454D503A0000000087
:208BC00000000053455041524154494F4E3A000000000000534B594C4C455449443A000076
:208BE00000000000004E4956454155205641534B3A00000000004E495645415520534B593F
:208C00004C3A000000000056454E54494C2E5449443A000000000000544F5252454D49444D
:208C200044454C0000000000004B4C4152204F56524947453F202020200050524F475241BF
:208C40004D204F2E4B2E3F20202000454E474C4953483F2020202020202020004445555497
:208C60005343483F2020202020202020004652414E434149533F20202020202020005356C8
:208C8000454E534B413F20202020202020200053554F4D493F202020202020202020200017
:208CA0004E454445524C414E44533F2020202020004954414C49414E4F3F202020202020A5
:208CC00020004E4F52534B3F2020202020202020202000455350414E4F4C3F202020202077
:158CE0002020200044414E534B3F20202020202020202020002F
:20B0000018CE6002BD954BBD954B18CE6002181D00A0181C00408630BD93F28630BD93F22D
:20B020008630BD93F28620BD93F28628BD94AFBD954B8606BD94AFBD954B8614BD94AFBD65
:1BB04000954B860CBD94AFBD954B8601BD94AFBD954B18CE6002181C002039ED
:20FF000001010A141E28323C46505152535455565758595AFF01010A141E28323C3D3E3F93
:20FF200040414243444546FF0A141E28323C000A0F14191E23282D32373C00000000010396
:14FF400000010600000300000000FF00010F1E2D3C4B5AFF69
:20FD0000DD8EDF9018DF92135002107F005CBDEB692608BDEB6F26031550021350400B7C20
:20FD2000007A967A810F2E0D20177A007A967A81002702200C135040051550402003145089
:20FD4000401350010EBDEAE67C008C968C81072E07200B7F008C2006BDEB62155001134F4F
:20FD600020037C005D134F40037C005E134F10037C005C7C0063860A91632E33134D800512
:20FD8000DE5708DF577C0079144E107C00597C005B7C00667C0067134F8007DC5FC3000130
:20FDA000DD5F7C005A7F0063134F02037C0078966427087A00642603154E04966527087AB9
:14FDC00000652603154E088640B71025DC8EDE9018DE923BE9
:20E000008600B710248693B710397F10358683B71026863EB710098E00FF8600B760018677
:20E02000FFB760008604B760018600B7600386E0B760028604B76003BD941118CE01F4BD6B
:20E0400093AEBDF678861497DF7F00327F00457F0046BDF762BDF13CBDF678BDF817BDE96D
:20E06000C2BDE994BDED1DB6103181FF27037EE084BDED4FB6103281FF27037EE084BDF62A
:20E08000787EA13886009727978DBD9309BDEB7B2700BDEB6F2706154E407EA0007EE285BC
:20E0A000154E41BD9309CCC096BD9343DC3FBD92F1BD931FCCC0A2BD9343DC41BD92F1CCFA
:20E0C000C119BD9343BD96AE124C01F9BD9309B6B715978BB6B714978A972CCCC0C0BDEF20
:20E0E000EE978ACEB714BD967B968B972CCCC0CFBDEFEE978BCEB715BD967B18CE01F4BDAF
:20E1000093AEBD9309BD931FCCC050BD9343BD930086019722BDEBFD962BBD92D1CCC113D1
:20E12000BD9343BD930086079722BDEC35962BBD92D1CCC113BD9343BD9300860D9722BD6B
:20E14000EC6D962BBD92D1CCC113BD9343BDE687965127037EE5CEBDEB6F261E20B0BD936B
:20E1600009CCC061BD9343BD931FCCC27BBD9343BD96AE124C01037EE252145001BD930041
:20E18000CCC085BD9343BD931FCCC27BBD9343BD96AE124C01E1BD9300CCC215BD9343BD4C
:20E1A0009300CEB7E0A600BD92D1CCC0E6BD9343CEB7E0A601BD92D1CCC0E6BD9343CEB7E6
:20E1C000E0A602BD92D1CCC0E6BD9343CEB7E0A603BD92D1CCC0E6BD9343CEB7E0A604BD93
:20E1E00092D1BD96AEBD9300CCC215BD9343BD9300CEB7E0A605BD92D1CCC0E6BD9343CEE2
:20E20000B7E0A606BD92D1CCC0E6BD9343CEB7E0A607BD92D1CCC0E6BD9343CEB7E0A6084C
:20E22000BD92D1CCC0E6BD9343CEB7E0A609BD92D1BD96AEBD9300CCC215BD9343BD9300AE
:20E24000CCC13DBD9343BD96AE124C01058663BDF215BD9309CCC1E2BD9343BD931FCCC2F7
:20E260007BBD9343BD96AE124C01048601978DBD9300CCC01BBD9343BD96AE124C01037E16
:20E28000F3F37EE0A0155002BDF817144E40BDF678BD930996339752963497537F005714F1
:20E2A0004D80BDEAFBCC00051A93572EF8BDEAFB154D80154E03154E01BDE90596512703EA
:20E2C0007EE5CEBDEBFD2646154E30BD9300CCC18DBD9343BD931FCCC19EBD9343BD96AE3E
:20E2E000124C01F9BDE9638602915127D68601915127C3144E30BD9309BD931FCCC1AFBDB0
:20E300009343144E32BDE83D8601915127A8144E0386019745144E30BDE9057F005714503A
:20E3200004144D80BD931FCCC1C0BD9343BD96AE124C01F9155004BDE905965127037EE6C7
:20E340005C155080144E30BD931FCCC215BD9343BD931FCCC111BD934396459645BD92D1CF
:20E36000CCC113BD9343BDE610967BBD92D1CCC0FFBD9343CCC113BD93439654810027069D
:20E38000CCC15FBD9343CC0000DD57145008144D80BD96AE124C020F7C0045963591452CB3
:20E3A000A086019745209A155008154D802000BD931FCCC215BD9343144E30145080BDE673
:20E3C000107F00577F0058144D80BDE687965127037EE5CECC00031A93572EEEBDE96396A5
:20E3E0005127037EE5CE18CE07D0BD93BFBDE83D965127037EE341CC0000DD57BDEABCBDF0
:20E40000EAD1BDE687965127037EE5CEBDEEE4CC000B1A93572EEBBDEAB5BDE687965127BE
:20E42000037EE5CEBDEEE4CC00161A93572EEBBDEAAECCC168DD7C144E80BDE6879651275D
:20E44000037EE5CEBDEEE4CC001B1A93572EEB4F91542703BDEACABDE687965127037EE588
:20E46000CEBDEEE4CC001BD3551A93572EE9BDEB2CBDE687965127037EE5CEBDEEE4CC007A
:20E480001BD355D3881A93572EE7154D80BDEB1018CE01F4BD93AEBDEB1718CE01F4BD9368
:20E4A000AEBDEB1E18CE01F4BD93AEBDEB3318CE01F4BD93AEBDECE12615BD931FCCC21584
:20E4C000BD9343154E80BD931FCCC14EBD9343BDE687965127037EE5CE7A00537A0053BD26
:20E4E000ECE1270220087C00537C005320E17C00537C0053BDEAC318CE01F4BD93AEBDEAD7
:20E50000D8144D80CCC172DD7C144E80BDE687965127037EE5CEDC86C3001BD355D3881ABF
:20E5200093572EE8BDEB2518CE01F4BD93AEBDEB47DC391A8300002725CCC000DD7CBDEABC
:20E54000A0BDE687965127037EE5CEDC86C30028D355D388D3391A93572EE6BDEB02968DEE
:20E5600081012724154D80154E80BD931FCCC215BD93437F00577F0058144E30155080BD83
:20E58000EF71BDE9057EE341BDEF71154EB0BD931FCCC215BD9343BD9309BDE905CCC16800
:20E5A000DD7CCCC1E2BD9343144D807F00577F0058BDE687965127037EE5CEBDEB6F2608C1
:20E5C000CC02321A93572EE9BD93097EE3AF8601915126037EE2B68602915126037EE2C359
:20E5E0008607915126037EE341860A915126037EE285860B915126037EF25D860C9151265E
:20E60000037EE0A0860D915126037EF0257EEA7F9645C6033DC300A38FA600975408A600CC
:20E62000977B972BC6B73DDD559637C6033DDD88D355DD7E9636C6033DDD86D37EDD7E96E8
:20E6400038498102270BC6033DDD39D37EDD7E2005CC000020F3C30028DD7E39BDE994BD42
:20E66000EADFBD9300BD931FCCC204BD934318CE01F4BD93AEBD931FCCC215BD934318CE89
:20E6800001F4BD93AE20DBBDEE49134E2007134E1003BDEDB2BD92AA134E0128BDEC6D2681
:20E6A00023860F91662E20BD9300154E30CCC226DD6DBD93438605BDF215154E01BDEA1D72
:20E6C000BDE65C397F0066BDEB872657BDEB812652BDEB6F2742124F0149144F10860A9111
:20E6E0005C2E46BDE9C2BDE994144F01BDE994154E80BDEB872603154E0C144E30BD930975
:20E70000BDE905154F01134E010586079751398601975139270920B9BDEB69270620B727E7
:20E720000220AE154F107F005C7A0052BDEC6D271DBDECA52618BDEBF126137C00527A00EE
:20E74000527A0052BDECA5260DBDEA8B20087C0052BDEAED20067C00527C00527A0053BD12
:20E76000EC352722BDECE1261D7C00537A00537A0053BDECE12617BDEBDF2612BDEBF726AE
:20E780000DBDEA9220087C0053BDEAF420067C00537C0053BDEB9A271B124F081E144F0867
:20E7A000BD9309CCC248DD6DBD93438608BDF215BDEA1D39BDEBA7270220DEBDEB8D271B11
:20E7C000124F041E144F04BD9309CCC259DD6DBD93438609BDF215BDEA1D39BDEBB427025D
:20E7E00020DE134E0217BDEBF72612BDEC35260D144F80CC044C1A935F2E11201A154F8051
:20E800007F005F124F0227BDEB09202DBDEAA77F0078144F022022BDEB09BD9309CCC26AA4
:20E82000DD6DBD9343860ABDF215BDEA1D39860691782E05154F0220CE7F0051397F0061A5
:20E84000BDE6879651270139BDEC6D2709BDEBFD27047F005139BDECA5261B7A00537A0051
:20E8600053BDECE127087C00537C005320087C00537C005320CABDEC3527C5BDE687965163
:20E88000270139124F02F47F005B18CE03E8BD93AEBDEAC3963B2703BDEAD8BDE687965122
:20E8A000270139965B815B2E1BBDEBFD27ED7F0079BDE6879651270139BDEBFD27DD861976
:20E8C00091792EEDBDEB25124E0109BD931FCCC1AFBD9343BDEB477C0061860391612E2207
:20E8E000BDEC6D270B860A91612E17BDEBFD2612BD9300CCC1D1BD93438602BDF215BDEAF8
:20E9000034397EE840134E2007134E1003BDEDB2BDE6879651270139124E04E9124E08E580
:20E920007F0059BDE68796517F0051270139BDEB87270CBDEB812707BDEAFB7F005139BD9C
:20E94000EAFB861691592EDB2009BDE994BDE9C27EE65CBD9300CCC237BD93438607BDF2D4
:20E960001520E7BDEA997F005ABDE6879651270139BDEB872609BDEB8126047F005139BD79
:20E98000E68796512701398616915A2EE47F0051BDE9EA39BDEB09BDEB2CBDEB10BDEB2586
:20E9A000BDEAEDBDEAF4BDEAFBBDEB33BDEB47BDEB1EBDEB02BDEB17BDEB5BBDEB62154E1D
:20E9C00080397F00577F00587F005F7F00607F00617F00627F005D7F005F7F004C154D80EC
:20E9E000154E3C154FF015500C39BDE9C2BDE994BDE905BD931F964E84012717144E30CCB9
:20EA0000C1F3BD9343BD96AE124C01F9BD9309124E010586029751398607975139BDE9C2D8
:20EA2000BDE994BDE905154E03BD9300DC6DBD93437EE65CBDE9C2BDE994BDE905154E33BC
:20EA4000BD931FCCC17CBD9343BD96AE124C01F9BD93098601975139BDE9C2144F01BDE9DF
:20EA600094154F01BDE905BD96AE124C01F9BD9309124E010586029751398607975139BDC6
:20EA80009300CCC02CBD93437EE65CCE60001C000839CE60001C000439CE60001C00023941
:20EAA000CE60001C000139CE10081C000239CE10081C000439CE10081C001039CE10081C09
:20EAC000000839CE10081C002039CE10001C008039CE10001C004039CE10001C002039CE53
:20EAE00010001C001039CE10001C000839CE60001D000839CE60001D000439CE60001D0007
:20EB00000239CE60001D000139CE10081D000239CE10081D000439CE10081D001039CE108D
:20EB2000081D000839CE10081D002039CE10001D008039CE10001D0040124F0109865B9741
:20EB4000659764144E0439CE10001D0020124F0109865B97659764144E0839CE10001D00BA
:20EB60001039CE10001D000839B66002841039B66002840839B66002840439B660028402D7
:20EB800039B66002840139B6100A848039B6100A84402703860039860139B6100A84202781
:20EBA00003860039860139B6100084042703860039860139B6100084022703860039860120
:20EBC00039B61000840139B66000840839B66000840439B61000844039B61000842039B6AA
:20EBE0001008840239B61008840439B61008841039B61008840839B610088420398603B796
:20EC0000103018CE0001BD93AECE10301E00800586019748397F0048F6103486C43DCE0029
:20EC200032028FCE000A028F17972B913D2E038600398601398602B7103018CE0001BD939B
:20EC4000AECE10301E00800586019748397F0048F6103386C43DCE0032028FCE000A028F35
:20EC600017972B913E2E038600398601398604B7103018CE0001BD93AECE10301E00800525
:20EC800086019748397F0048F6103186C43DCE0032028FCE000A028F17972B913D2E0386F8
:20ECA00000398601398600B7103018CE0001BD93AECE10301E00800586019748397F0048E2
:20ECC000F61031C02C86413DCE0095028FCE0001028F1780059B8A91522E0386003986019E
:20ECE000398601B7103018CE0001BD93AECE10301E00800586019748397F0048F61032C069
:20ED00002C86413DCE0095028FCE0001028F1780059B8B91532E038600398601398600B7DC
:20ED2000103018CE0001BD93AECE10301E00800586019748397F0048F61031C02C86413D70
:20ED4000CE0095028FCE0001028FC005DB8A398601B7103018CE0001BD93AECE10301E006D
:20ED6000800586019748397F0048F61032C02C86413DCE0095028FCE0001028FC005DB8B01
:20ED80003997987F0097BD95CF8620BD9620CE009DA60081202704BD953B390820F3DD9789
:20EDA000BD95CF8620BD9620CE009D20E4BD953B3939134E20FBBDEBC7270413504019BD1C
:20EDC0009300BD930086019722BDED1D17BD92D1CCC0FCBD93432016BD9300BD930086019A
:20EDE0009722CCC0F9BD9343CCC0F9BD9343BDEBCD270413504016BD9300860B9722BDED8D
:20EE00004F17BD92D1CCC0FCBD93432013BD9300860B9722CCC0F9BD9343CCC0F9BD934354
:20EE200013508016BD930086079722CCC111BD93439645BD92D1154E1039BD9300860797F7
:20EE400022CCC0F9BD934320ED134E8056BD931FDC7CBD9343DC7E93570C59490C59490C2E
:20EE600059490C59490C5949CE0064028FDD80CE003C028FD782863C3DDD83DC809383D7D8
:20EE8000859682BD92D1CCC0E2BD9343968581092E06CCC115BD93439685BD92D1CCC0DE01
:20EEA000BD9343398FBD953B393C183C3637200CC61086104A26FD5A26F82005BDEB6F2754
:20EEC000FB3332183838393C183C3736BD93093233183838393C183C3736BDEB6F27FB322D
:20EEE0003318383839BD9300BD931F9657BD92F1398600CEB709BD967B8600CEB70908BD3E
:20EF0000967B8600CEB711BD967B8600CEB71108BD967B8600CEB713BD967B8600CEB716F7
:20EF2000BD967B8600BDF2158600BDF2158600BDF2158600BDF2158600BDF2158600BDF25C
:20EF4000158600BDF2158600BDF2158600BDF2158600BDF2158603CEB721BD967B8608CE1B
:20EF6000B722BD967BBD9309CCC0AEBD93437EEF6EB6B7169744FCB709DD3FFCB711DD41D1
:20EF8000B6B71397439B7B813B2E569743DC3FC30001DD3F96449B37813B2E02200C803C6C
:20EFA000974496438B019743964497449643CEB713BD967B9644CEB716BD967BDC41CEB75E
:20EFC00011BD967BDC4117CEB71108BD967BDC3FCEB709BD967BDC3F17CEB70908BD967BA5
:20EFE00039803C9743DC41C30001DD41209FDD6DBD9300DC6DBD9343962C81092E06CCC101
:20F0000013BD9343962CBD92D1BD96AE124C0212962C8B01972C81142E0220D48601972CE1
:20F0200020CE962C39154E40BDF817BD9300BD931FCCC0F9BD9343BDEB692708CCC0E6BD32
:20F0400093432003BDF132BDEB6F2708CCC0E6BD93432003BDF132BDEB752708CCC0E6BD0E
:20F0600093432003BDF132BDEB7B2708CCC0E6BD93432003BDF132BDEB812708CCC0E6BDD6
:20F0800093432003BDF132BDEB872708CCC0E6BD93432003BDF132BDEB8D2608CCC0E6BD9F
:20F0A00093432003BDF132BDEB9A2608CCC0E6BD93432003BDF132BDEBA72608CCC0E6BD53
:20F0C00093432003BDF132BDEBB42608CCC0E6BD93432003BDF132BDEBC12708CCC0E6BDFE
:20F0E00093432003BDF132BDEBFD962BBD92D1CCC113BD9343BD930086079722BDEC359674
:20F100002BBD92D1CCC113BD9343BD9300860D9722BDEC6D962BBD92D1CCC113BD9343BDEE
:20F12000EB6F26037EF02BBDEB6F26FBBD93097EF127CCC115BD9343397EF1D9963C972845
:20F1400086099729BDF20726F09635972886099729BDF20726E396349728865A9729BDF224
:20F160000726769633972886469729BDF207266996379728863C9729BDF207265C963697EA
:20F1800028863C9729BDF207264F963D9728865A9729BDF2072642963E9728865A9729BD5A
:20F1A000F207263596389728865A9729BDF2072628963B972886019729BDF207261B968ADC
:20F1C000972886149729BDF207260E968B972886149729BDF207260139BDF7CF860A978AA8
:20F1E000978BBDF6E7968ACEB714BD967B968BCEB715BD967B8603973CCEB706BD967B8608
:20F2000062BDF2157EE65C9628912922022003860139860039CEB7E0E600BD967B0817E6AC
:20F2200000BD967B0817E600BD967B0817E600BD967B0817E600BD967B0817E600BD967BB4
:20F240000817E600BD967B0817E600BD967B0817E600BD967B0817E600BD967B39BD931FBA
:20F26000CCC27BBD9343BDF817154E027F0032BD9300BDF511BD96AE124C0208BDF520BD05
:20F28000F67820D9BDF678BD931FCCC27BBD9343BD9300CCC28CBD9343BD96AE124C01165E
:20F2A000BD9300CCC29DBD9343BD96AE124C0106BDF7CF7EF40A7C0032BD9300CCC215BD7D
:20F2C0009343BD9300CCC29DDD6BBDF426BD96AE124C0205BDF52020E086019745BD9300D3
:20F2E000CCC111BD93439645BD92D18603D6453DC300A3C30000DD2E8FA60081FF26048668
:20F3000000A70081002708CCC103BD93432006CCC10ABD9343CCC15FBD9343BD96AE124C45
:20F320000210DE2E6C008602A10026026F00DF2E20ABBD9300CCC111BD93439645BD92D12F
:20F34000CCC2BFBD93438603D6453DC300A3C30001DD2E8FA60081FF26048601A700BD925B
:20F36000D1CCC0FFBD9343BD96AE124C0210DE2E6C008609A1002ABA8601A70020B47C0023
:20F380004596358B01914527037EF2DD7C0032BD9309BD931FCCC27BBD9343BD9300CCC294
:20F3A000D0BD9343BD96AE124C015FBD9300CCC215BD9343BD9300CCC2BFDD6BBDF426BD2C
:20F3C00096AE124C0205BDF52020E97C0032860991322AD77F0032BD9300CCC00ABD93437E
:20F3E000BD931FCCC27BBD9343BD96AE124C01037EE0A0BD9300CCC369BD9343BD96AE12B3
:20F400004C0207860297327EF3B4BD9300CCC37ABD9343BD96AE124C02037EF25DBDF6E76A
:20F42000BD93097EE285BD931FCCC27BBD9343BD93008611D6323DD36BBD9343860191323C
:20F4400026059635BD92D1860291322617963481012606CCC113BD93439634BD92D1CCC0ED
:20F46000FCBD9343860391322617963381012606CCC113BD93439633BD92D1CCC0FCBD9309
:20F480004386049132260B9637BD92D1CCC04EBD934386059132260B9636BD92D1CCC04E0C
:20F4A000BD9343860691322611963DBD92D1CCC117BD9343CCC0F9BD93438607913226116A
:20F4C000963EBD92D1CCC117BD9343CCC0F9BD934386089132262196384981022712BD922F
:20F4E000D1CCC04EBD9343CCC0F9BD93437EF4F8CCC115BD934320E9860991322612963BB3
:20F500002708CCC103BD93432006CCC10ABD934339BD93008611D63C3DC3C38BBD934339FD
:20F520008600913226127C003CBDF6788609913C2A6F7F003C7EF6748601913226107C00D3
:20F5400035860991352A5A860197357EF6748602913226237F0068CCFF008FD6683AA6006F
:20F5600081FF26067F00687F003491342E057C006820E49734202A8603913226277F0068D0
:20F58000CCFF158FD6683AA60081FF26067F00687F003391332E057C006820E497337EF67C
:20F5A000747EF6748604913226247F0068CCFF288FD6683AA600810026067F00377F006887
:20F5C00091372E057C006820E497377EF6748605913226237F0068CCFF2F8FD6683AA6006D
:20F5E000810026067F00687F003691362E057C006820E49736207D860691322613963D8B90
:20F600000A973D8663913D2A6B860A973D7EF674860791322613963E8B0A973E8663913EF5
:20F620002A52860A973E7EF6748608913226237F0068CCFF4B8FD6683AA60081FF26067F92
:20F6400000687F003891382E057C006820E49738202286099132260F963B27057F003B2038
:20F66000138601973B200DCCC02CBD934318CE03E8BD93AEBDF80D39963C81002607CCC4CC
:20F6800060DD69206181012607CCC8C0DD69205681022607CCCD20DD69204B81032607CCED
:20F6A000C000DD69204081042607CCD180DD69203581052607CCD5E0DD69202A8106260702
:20F6C000CCDA80DD69201F81072607CC8000DD69201481082607CC8460DD6920098109267F
:20F6E00005CC88C0DD69399633CEB700BD967B9634CEB701BD967B9635CEB702BD967B9682
:20F7000036CEB703BD967B9637CEB705BD967B963CCEB706BD967B963DCEB707BD967B964A
:20F720003ECEB717BD967B9638CEB719BD967B963BCEB720BD967B963FCEB709BD967B96DC
:20F7400041CEB711BD967BBDF80DC600CEB60018CE00A318A600BD967B0818085CD1472621
:20F76000F239B6B7009733B6B7019734B6B7029735B6B7039736B6B7059737B6B706973CF0
:20F78000B6B707973DB6B717973EB6B7199738B6B720973BFCB709DD3FFCB711DD41B6B7ED
:20F7A000139743B6B714978AB6B715978BB6B7169744BDF13CBDF80DC600CEB60018CE00DC
:20F7C000A3A60018A7000818085CD14726F339863C973386559734860397358614973686BF
:20F7E0001E97378628973D860A973E860197388600973BBDF80DC600CEFF3B18CE00A3A6C9
:20F800000018A7000818085CD14726F3398603D6353DCB03D7473918CE012CBD93AE7F00B5
:1FF820005018CE1024181C0040BDE9C2154FFF154E801450408600977A0E18CE00C8390D
:209200009626810F2E0786809B267E921186B09B26BD95218600B76001860FB760008604A7
:20922000B7600118CE6002181C0020181C0040181C0080B6600084F0972418CE6002181D90
:209240000080181C0080B6600084F09725181D00E08600B7600186FFB760008604B76001A3
:20926000962546464646840F9A24972439A600271A3696238101260732BD93757E92833295
:20928000BD93920886194A26FD20E2399626810F2E0ACC0000DB26188F7E92A6CC0011DB37
:2092A00026830010188F18A60039BD9200BD928C9124260F96264C9726811F2E01398600F0
:2092C000972639BD9411BD94DDBD9328860097263997987F0097BD95CF8620BD9620CE00C7
:2092E0009DA60081202707BD926DBD9328390820F0DD97BD95CF8620BD9620CE009D20E1BD
:20930000860197238600972239BD9300CCC215BD9343BD931FCCC215BD9343BD930039865A
:209320000297238600972239BD932FBD933939BD9505CC0000BDEEA439BD94FFCC0011BD23
:20934000EEA43983C000D3698FA600810027183C3696238101260732BD93757E936232BD9B
:20936000939238087E9349962381012604BD932F39BD93393918CE0000D622C100270BC1BD
:20938000112E0E18085AC10026F918A7007C0022393918CE0011D622C100270BC1112EF184
:2093A00018085AC10026F918A7007C002239183C3CCE01470926FD38180926F418383918D7
:2093C0003C3CCE01470926FD38180926F4183839183C3CCE00200926FD38180926F418386A
:2093E0003936B66000840F972D3284F09A2DB760003918CE6002181D0040BD93E118CE60A0
:2094000002181C0080181D0080181C0040BD954B3918CE6002BD954BBD954B18CE600218B5
:209420001D00A0181C00408630BD93F28630BD93F28630BD93F28620BD93F28628BD94AF7D
:20944000BD954B8606BD94AFBD954B8614BD94AFBD954B860CBD94AFBD954B8601BD94AF59
:20946000BD954B18CE6002181C002018CE6002181D0020181D00408640BD94AFBD954B1826
:20948000CE6002181C0020CE958FDF6D8640972BDE6DA60008DF6DBD94AFBD954B962B4A95
:2094A000972B810026EA18CE6002181C00203918CE6002973184F0BD93E1BD94CC96318467
:2094C0000F48484848BD93E1BD94CC39181D0040181C0080181D0080181C00403918CE6005
:2094E00002181D00208601BD94AFBD954BBD954B18CE6002181C0020398680BD9521398647
:20950000C0BD95213918CE6002181D00208602BD94AFBD954BBD954B18CE6002181C0020E4
:209520003918CE6002181D0020BD94AFBD954BBD954B18CE6002181C002039A600270BBDB1
:2095400094AF0886194A26FD20F13918CE0014BD93AE3936375F8164251A5C806481642400
:20956000F9CB303617BD94AF325F810026068630BD94AF4F810A250F5C800A810A24F9CB4F
:20958000303617BD94AF328B30BD94AF33323904000E111F1111000A001F111F1111000ADA
:2095A000000E1111110E0003041F101E101F0002051F101E101F0003041F111F11110011CD
:2095C00000111111111F000E11101010150E037F00947F00957F00968610979ACE009686C6
:2095E000039799A600979B840F80052B06969B8B03979B969B84F080502B06969B8B3097FD
:209600009B969BA700097A009926D87800987900977900967900957900947A009A26BD3943
:20962000CE009DA700088C00A126F8CE00009694840F27058B30979D0896954444444426B6
:2096400006D69DC12027058B30979E089695840F2606D69EC12027058B30979F08969644B8
:209660004444442606D69FC12027048B3097A09696840F8B3097A17F00A23937183CC6160C
:20968000F7103BE700C617F7103B18CE000ABD93AE7F103BC602F7103BA700C603F7103B0E
:2096A00018CE000ABD93AE7F103B1838333936373C183C154C03BDEB6926FBBDEB6F26F670
:2096C00018CE0019BD93AEBDEB6926EABDEB6F26E5134E4003BDE687BD92AABD971ABDEB6D
:2096E0006927037E96FFBDEB6F27E618CE0019BD93AEBDEB6F27DA144C0214500220121879
:20970000CE0019BD93AEBDEB6927C6144C01145002145001183838333239134E2007134E2B
:069720001003BDEDB2399B
:20A00000BDA101BD930986009730BD9300CCC03DBD93439630BD92D1BD931FCCC27BBD93E1
:20A0200043BD96AE124C01037EA03E7C00309630810A27037EA00A860097307EA00ACC008E
:20A0400000DD2EBD9300CCC03DBD93439630BD92D1DC2EBD92F1BD931FCCC27BBD9343BD51
:20A0600096AE124C01037EA081DC2EC30001DD2E1A83000A27037EA043CC0000DD2E7EA09B
:20A08000439630B1B7212617962FB1B72226102007860C97517EE5CE860B97517EE5CEBD33
:20A0A000930996308107260ADC2E1A83000226022007860A97517EE5CE86009730BD930048
:20A0C000CCC03DBD93439630BD92D1BD931FCCC27BBD9343BD96AE124C01037EA0F17C0045
:20A0E000309630810A27037EA0BD860097307EA0BD9630810926BBBD9309860D97517EE54A
:20A10000CEBDEB6F26FBBD9300CCC0E8BD9343BD931FCCC27BBD9343CC0000DD57144D80F6
:20A12000DC571A83000A2E05BDEB6927037EA0B2BDEB6F27EB7EA003BDF817BDF678860040
:20A140009727154E40BD9309CCC11BBD9343B6B721BD92D1B6B722BD92D1BD931FCCC27B35
:20A16000BD9343BD96AE124C01037EA1707EA1FEBD930986009730BD9300CCC03DBD9343EB
:20A180009630BD92D1BD931FCCC27BBD9343BD96AE124C01037EA1AB7C00309630810A277D
:20A1A000037EA177860097307EA177CC0000DD2EBD9300CCC03DBD93439630BD92D1DC2EB0
:20A1C000BD92F1BD931FCCC27BBD9343BD96AE124C01037EA1EEDC2EC30001DD2E1A83004E
:20A1E0000A27037EA1B0CC0000DD2E7EA1B09630CEB721BD967B962FCEB722BD967BBD93F2
:0AA2000009CCC12CBD93437EA207D8
:008000017F
